:100000000C9475000C9400000C9400000C940000FB
:100010000C9400000C9400000C9400000C94000060
:100020000C9400000C9400000C9400000C94000050
:100030000C9400000C9400000C9400000C94000040
:100040000C9400000C9400000C9400000C94000030
:100050000C9400001027E80364000A00010000105F
:1000600000011000010080C000002067617465205D
:1000700073696D756C61746F7220002020616C690A
:10008000202068657964617269202000616E6400D7
:100090006F7200786F72006E616E64006E6F720036
:1000A000786E6F72006E6F74006625693D2025734F
:1000B000206D6F64652000783D2569202C20793DF6
:1000C0002569202C20663D256900783D2569202082
:1000D00020202C20202020663D25690002006001A0
:1000E00066000200640168000000F894EE27ECBB93
:1000F000F1E0FBBFEBBFE5BFF8E1F1BDE1BD8DE095
:10010000A2E0BB27ED938A95E9F780E094E0A0E6B2
:10011000ED930197E9F7ECEDF0E08591959100976B
:1001200061F0A591B59105901590BF01F001059082
:100130000D920197E1F7FB01F0CFEFE5EDBFE4E0B1
:10014000EEBFC0E6D1E00C94A500A597E2E0FE2E3C
:1001500000E010E0E8E0EBBBEABBE0E0E2BBE0E49B
:10016000E1BBE0E1EA930E94F103EEE5F1E00E94D9
:100170003D04839B0EC0E4E6F0E00E943D04839BB7
:1001800002C00F5F1F4F0830E0E01E0714F007E0C9
:1001900010E0829B0EC0E4E6F0E00E943D04829BEA
:1001A00002C0015010400130E0E01E0714F401E0ED
:1001B00010E0F8013097A9F4F1FE12C00E948F03FD
:1001C000EAE6F0E0FA93EA930E94CE030E9441042B
:1001D000EBE7F0E0FA93EA930E94CE03E894F1F89B
:1001E00065C0E130A0E0FA0751F40E944704EA2319
:1001F0000E944F04ECE8F0E00E94560457C0E23041
:10020000A0E0FA0751F40E944704EA2B0E944F0431
:10021000E0E9F0E00E94560449C0E330A0E0FA07AC
:1002200051F40E944704EA270E944F04E3E9F0E0FA
:100230000E9456043BC0E430A0E0FA0751F40E944B
:100240004704EA230E945F04E7E9F0E00E945604B5
:100250002DC0E530A0E0FA0751F40E944704EA2BD4
:100260000E945F04ECE9F0E00E9456041FC0E630F3
:10027000A0E0FA0751F40E944704EA270E945F04B5
:10028000E0EAF0E00E94560411C0E730A0E0FA076F
:1002900069F4E894B09B6894F0F8FE01FA93EA934D
:1002A000E5EAF0E00E9456046894F2F8F1FE4DC0D1
:1002B000F0FAA2B3A6F9A2BB0E948F03FE017596C5
:1002C000FA93EA93E9EAF0E0FA93EA93F8010E94DC
:1002D000D3040E94E004FE013896662777270E9427
:1002E0006804FE017596FA93EA930E94BF030E9488
:1002F0004104F2FC16C00E946F04E7EBF0E00E949C
:100300007404E0E0B199E1E0FF27662777270E94B7
:10031000E0040E947F040E94E0048CE00E940A0333
:100320006096F2FE0CC00E946F04EAECF0E00E94BE
:1003300074040E947F040E946804E894F2F80E940A
:100340006F040E94BF03E894F1F80FCFFFCF5F9BCB
:10035000FECFECB108955D9BFECFE881ECB921960C
:1003600008951A930A93AC81BD810E94D8043097F6
:10037000D9F0AA81BB810E94D8048F01309749F03F
:100380000230E0E01E0778F0F80131978F01ED931D
:10039000FC93AC81BD81ED91FD913196FE93EE937E
:1003A0003197AE81A08304C0EE81EA930E94AB0135
:1003B000198108812796089526970E94EA0410E083
:1003C000EA89FB893196EA8BFB8B3197E4912E2FDA
:1003D000E03011F40C940603E12FE03039F42532BB
:1003E00011F411E002C00E9486040FC1E130A9F4AB
:1003F000253219F40E94860407C112E040E000E0B3
:100400002D3211F401E001C12B3211F44BE2FDC099
:10041000203211F440E2F9C002C0E23039F450E079
:1004200013E0203311F40068F0C004C0E33011F091
:100430000C940503203310F02A3308F009C0A52FCF
:10044000EAE0EA9FF0015E2FE22FE0535E0FDDC08D
:10045000E22FE33631F40E949104EC910E9498045B
:10046000D3C0E33741F40E9491040E94A3040E9488
:1004700028041E2F0AC0E03761F40E9491040E94F4
:10048000A3040E9432041E2F086002600F7730E040
:1004900038C0E43611F0E93611F4046002C0E537E3
:1004A00031F4E4E5F0E0EE83FF8315E00DC0E835BC
:1004B00011F4086004C0E83711F00C940403EEE571
:1004C000F0E0EE83FF8314E002FF15C00E94910468
:1004D0000E94D804EA87FB87AA85BB8510972CF475
:1004E0000E94CF04EA87FB874DE2403011F01F5F86
:1004F00001C00B7F06C00E9491040E94D804EA87C5
:10050000FB8700FD11C0151778F407FF08C002FF34
:1005100004C00B7F242F115001C020E301C020E252
:100520000E9486045150EFCF312F01FF1AC03030A6
:10053000B9F003FF08C0EE81FF813196EE83FF839F
:100540003197E49105C0AE81BF81ED91AE83BF8349
:10055000EA930E94AA04503009F051503150E7CF7D
:100560004AC020E3EE81FF813296EE83FF8332970B
:100570000E94DC04E887F987E885F985AA85BB85B0
:10058000AE17BF0750F02F5FA885B985EA85FB85B8
:10059000EA1BFB0BEA87FB87EFCF2A3328F003FF28
:1005A00002C0295F01C0295D04FD1AC0213320F477
:1005B000A885B985119709F409C0531710F000FFF9
:1005C00001C013C020E207FF0BC020E3006102FF5F
:1005D00007C00B7F4A930E94AA04503009F0515083
:1005E0000E948604503009F051503150A885B985D9
:1005F000129708F0B6CF00FF07C0503029F05150D5
:10060000E0E20E949804F9CF10E0DACE0E94F104F3
:1006100064960895FF92F82E22971A930A93DE01AA
:100620000E94CB048D01DE0116960E94CB040E942D
:10063000D804EA83FB83DE0114960E94CB040E9457
:10064000D804FA93EA931A930A93FE013696FA9322
:10065000EA93E0E0F0E0FA93EA930E94DC01AA81D9
:10066000BB81E0E0EC93198108812496FF90089506
:10067000FFE0FA95F1F70895AAB3AF70AABBD99A33
:10068000D8980E943803DA9A0E943803A9B3DA98FE
:100690000E943803DA9A0E943803DA98A7FDF1CF56
:1006A0000895A07FAB2BABBBDA9A0E943803DA988F
:1006B0000E9438030895D998AAB3A76FAABBBBB309
:1006C000BF70A8810E945103A881A2950E94510386
:1006D000D99A21960895DA9A0E943803E9B3DA98F4
:1006E0000E943803E07F08950E9438030E946B0344
:1006F000AE2F0E946B03D998E295EA2B08950E94D1
:100700003C03E881F0E0E05AFE4FE081A981EA0F66
:10071000EA930E945B0359804880229608950E94C4
:100720003C03E2E0EA930E945B030E943C03ECE09E
:10073000EA930E945B030E943C03E1E0EA930E947B
:100740005B03E0E04E2E5E2E0895EF93FF93A881A9
:100750006894AA3021F0E8945394751438F44394C3
:10076000E0E0EA934A920E947F032EF085DFD89A58
:10077000A881AA93A0DFFF91EF91219608951A9383
:10078000A981BA81ED91A983BA831E2FE03021F0AF
:100790001A930E94A503F4CF188110C01A93E9811F
:1007A000FA813196E983FA833197E4911E2FE03084
:1007B00021F01A930E94A503F2CF18812396089581
:1007C000AA27BB271197F1F70895D998AAB3A76F65
:1007D000AABBBBB3BF70A8810E945103D99A2196CE
:1007E0000895DA98D8987880E881E058E09362011B
:1007F000E881E054E09363010E94B4040E94B404D1
:100800000E94B4040E94E003E0E2EA930E94E50340
:100810000E94E003E8E20E94BA04E4E00E94BA0405
:10082000E5E80E94BA04AAB3AF70AABBD99A0E94A5
:100830007403E53011F0E0E009C00E943C03E6E0FB
:10084000EA930E945B030E948F03E1E021960895E2
:10085000A991B991EE27FF276D91662311F031968A
:10086000FBCF0895AA27BB27E991F99105900020B5
:1008700011F01196FBCFFD010895FA93EA930C94C1
:10088000BF04E0E0EA93E1E0EA930C947F03E0E048
:10089000B099E1E0AE2FE0E0B199E1E008950E9467
:1008A000E504F0F8FE01FA93EA930895FA93EA93C7
:1008B00080E00E940A0324966894F1F808950E944B
:1008C000E504F0F8E1E0FE26FE01FA93EA930895CC
:1008D0000E94E00488E00E940A032C960895FE011D
:1008E0003596FA93EA930895FA93EA93E0E0B09983
:1008F000E1E0FF27662777270E94E0040895E0E003
:10090000F0FCE1E0FF276627772708952A93EF851B
:10091000F889FA93EA93FE013F96FA93EA930C94CE
:10092000B101A889B9891497A88BB98B1496089539
:10093000EA93EF85F889FA93EA93FE013F96FA93DA
:10094000EA930C94B1010E94D804EE83FF83FA93DA
:10095000EA930895EF85F889FA93EA93FE013F96AA
:10096000FA93EA930C94B1010E94E003E0E3EA9366
:100970000C94E503EA930E945B030C94E003E99175
:10098000F991309639F080ED97E00197F1F7A8954D
:100990003197C9F708950024AF0DB01D0895F19562
:1009A000E195F04008956F2F660F660B762F08953E
:1009B000ED91FC91119708950590F491E02D089523
:1009C0007A936A93FA93EA930895E894EE2309F0F0
:1009D000689408955A934A933A932A931A930A93E0
:1009E00008955D814C813B812A8119810881089598
:00000001FF
